:020000040000FA
:040000008301C5288B
:08000800FF00030E8301A000BC
:100010000A08A1000408A2008A010313831222081F
:10002000B4002308B5002408B6002508B700260848
:10003000B8002708B9002808BA002908BB002A0818
:10004000BC002B08BD002C08BE002D08BF002E08E8
:10005000C0002F08C1003008C2003108C3003208B8
:10006000C4003308C5008B18C6283408A200350820
:10007000A3003608A4003708A5003808A6003908F0
:10008000A7003A08A8003B08A9003C08AA003D08C0
:10009000AB003E08AC003F08AD004008AE00410890
:1000A000AF004208B0004308B1004408B200450860
:1000B000B3002208840021088A00200E8300FF0E6E
:1000C0007F0E09002E08AC070318AF0A2F08AD07F2
:1000D00000342F08A3002E08A400A501A6011030AB
:1000E000AB00A40DA30DA60DA50D24102C08A8008F
:1000F0002D08A7002608A9002508AA002808A6029E
:100100000318852803198528A70A2708A5020318BC
:100110009E2803199E282908A6002A08A500A40DD8
:10012000A30DA60DA50D2410AB0B76280310A50C6E
:10013000A60C2308AD002408AC000034A40DA30DC8
:10014000A60DA50D2414AB0B76280310A50CA60C48
:100150002308AD002408AC0000342C08300203183A
:10016000B6280319B6280130B0000034B0010034BD
:100170002F082D02031DC3282E082C02031DC3289F
:100180000130B0000034B0010034CE2803138312D4
:100190000130C8070318C70A8B10352803138312D0
:1001A0000030831685000130860021308312AE00B6
:1001B000F830AD00B930AC00AC0BDC28AD0BDA2860
:1001C000AE0BD8284430B100B10BE4280000000089
:1001D000C801C701C60101170B170B168B170B17A8
:1001E0009101FF3083169200003083129500970131
:1001F0000F3097040030970483168611831212156E
:1002000083168C100313831610308312AE007330E4
:10021000AD00CE30AC00AC0B0B29AD0B0929AE0BF9
:1002200007291330B100B10B1329000000000000B2
:100230004808AC004708AD002C08B2002D08B300F8
:100240000030AC000030AD003308AF003208AE0023
:10025000B820031383120130B0063008301C7B290C
:100260004808AC004708AD002C08B2002D08B300C8
:100270000230AC000030AD003308AF003208AE00F1
:100280006920031383122C08CA002D08C9004A08EC
:10029000F63986004A08093985004808AC00470845
:1002A000AD002C08B2002D08B3000030AC000130C6
:1002B000AD003308AF003208AE0062200313831292
:1002C0002C08C8002D08C70047080339C7000339A8
:1002D0004708AD004808AC002C1817161712AC18C8
:1002E00097169712AD0CAC0CAD0CAC0C2C0895000D
:1002F000C801C7019C2903138312C60A4608B2002D
:100300000230B0003208AC00AD2003138312300875
:10031000301C9A29C601003085000030860000306C
:1003200095000F309705003097048316061183124D
:0E033000C801C70103138312031383120229AD
:00000001FF
